:020000040000FA
:10000000BB0A03040F0328000304080328008F0021
:100010002D008B000D0203062B00030428030304AC
:1000200008032E008B000E0203072B000008070CAC
:10003000810143070008E9044607E905000817099C
:10004000AB0C81000306000866071F0A1709AB0CFA
:100050008100030600086606260A750C8100030766
:100060001F0A0304010361002F0003040008E906CE
:100070005A0A26065A0A0907470A2907470A49075A
:10008000450A080C8907A901470A400CA90109047F
:1000900029040008A9020907000829070008C90661
:1000A000560A0E0289062B00A9062B004904080CEB
:1000B0002A00000809074A0A29074A0AEA004307F2
:1000C000000849066E0AC9066B0A0D0289062B0054
:1000D000A9062B00C9054905050C580A0D028B011C
:1000E000430669050E028B01430669046906EB00AD
:1000F0006907AB02030C580A0D02C907850AEC0018
:10010000EC000C028B000B0203062C000008890493
:10011000A9040F0C06002F0CA606910A06008905FB
:1001200000081E0C26002F0CA607980A0600A90539
:1001300006003E0C260000080A0C28002E0C2600A3
:100140002E0C0600A30AA40AA50AA60A3E0C260045
:100150002F0C0600E80043079E0A000817090C024E
:1001600081014307AE0A9C0A17090C02CF018101E5
:100170004307B40A9C0AC60C02003E0C26002F0C52
:1001800006006A006800E8004307C30AEA00430764
:10019000C30A69006607CA0A6606CC0A61008709B5
:1001A0001F0901090E022B001F090306CA0A87094D
:1001B000370901097C09C907D40AAE09B409D40A70
:080400000100000000000600ED
:021FFE00EA0FE8
:00000001FF
